 WinFallbackLookup

 Timestamp is c513c980 (reproducible build file hash)

 Preferred load address is 10000000

 Start         Length     Name                   Class
 0001:00000000 00001b8bH .text$mn                CODE
 0002:00000000 000000acH .idata$5                DATA
 0002:000000ac 00000008H .00cfg                  DATA
 0002:000000b4 00000004H .CRT$XCA                DATA
 0002:000000b8 00000004H .CRT$XCZ                DATA
 0002:000000bc 00000004H .CRT$XIA                DATA
 0002:000000c0 00000004H .CRT$XIZ                DATA
 0002:000000c4 00000004H .CRT$XPA                DATA
 0002:000000c8 00000004H .CRT$XPZ                DATA
 0002:000000cc 00000004H .CRT$XTA                DATA
 0002:000000d0 00000008H .CRT$XTZ                DATA
 0002:000000d4 00000000H .gfids$y                DATA
 0002:000000d8 00000168H .rdata                  DATA
 0002:00000240 00000000H .rdata$CastGuardVftablesA DATA
 0002:00000240 00000000H .rdata$CastGuardVftablesC DATA
 0002:00000240 00000004H .rdata$sxdata           DATA
 0002:00000244 0000005cH .rdata$voltmd           DATA
 0002:000002a0 000002a8H .rdata$zzzdbg           DATA
 0002:00000548 00000004H .rtc$IAA                DATA
 0002:0000054c 00000004H .rtc$IZZ                DATA
 0002:00000550 00000004H .rtc$TAA                DATA
 0002:00000554 00000004H .rtc$TZZ                DATA
 0002:00000558 00000088H .xdata$x                DATA
 0002:000005e0 00000050H .edata                  DATA
 0002:00000630 00000064H .idata$2                DATA
 0002:00000694 00000014H .idata$3                DATA
 0002:000006a8 000000acH .idata$4                DATA
 0002:00000754 00000414H .idata$6                DATA
 0003:00000000 000000f0H .data                   DATA
 0003:000000f0 00000374H .bss                    DATA
 0004:00000000 00000060H .rsrc$01                DATA
 0004:00000060 00000350H .rsrc$02                DATA

  Address         Publics by Value              Rva+Base       Lib:Object

 0000:00000000       ___AbsoluteZero            00000000     <absolute>
 0000:00000000       ___arm64x_extra_rfe_table  00000000     <absolute>
 0000:00000000       ___arm64x_extra_rfe_table_size 00000000     <absolute>
 0000:00000000       ___arm64x_native_entrypoint 00000000     <absolute>
 0000:00000000       ___arm64x_redirection_metadata 00000000     <absolute>
 0000:00000000       ___arm64x_redirection_metadata_count 00000000     <absolute>
 0000:00000000       ___dynamic_value_reloc_table 00000000     <absolute>
 0000:00000000       ___enclave_config          00000000     <absolute>
 0000:00000000       ___guard_check_icall_a64n_fptr 00000000     <absolute>
 0000:00000000       ___guard_eh_cont_count     00000000     <absolute>
 0000:00000000       ___guard_eh_cont_table     00000000     <absolute>
 0000:00000000       ___guard_fids_count        00000000     <absolute>
 0000:00000000       ___guard_fids_table        00000000     <absolute>
 0000:00000000       ___guard_iat_count         00000000     <absolute>
 0000:00000000       ___guard_iat_table         00000000     <absolute>
 0000:00000000       ___guard_longjmp_count     00000000     <absolute>
 0000:00000000       ___guard_longjmp_table     00000000     <absolute>
 0000:00000000       ___hybrid_auxiliary_delayload_iat 00000000     <absolute>
 0000:00000000       ___hybrid_auxiliary_delayload_iat_copy 00000000     <absolute>
 0000:00000000       ___hybrid_auxiliary_iat    00000000     <absolute>
 0000:00000000       ___hybrid_auxiliary_iat_copy 00000000     <absolute>
 0000:00000000       ___hybrid_code_map         00000000     <absolute>
 0000:00000000       ___hybrid_code_map_count   00000000     <absolute>
 0000:00000000       ___hybrid_image_info_bitfield 00000000     <absolute>
 0000:00000000       ___x64_code_ranges_to_entry_points 00000000     <absolute>
 0000:00000000       ___x64_code_ranges_to_entry_points_count 00000000     <absolute>
 0000:00000001       ___safe_se_handler_count   00000001     <absolute>
 0000:00000100       ___guard_flags             00000100     <absolute>
 0000:00000000       ___ImageBase               10000000     <linker-defined>
 0001:00000000       _vswscanf                  10001000 f i WinFallbackLookup.obj
 0001:00000020       _vswscanf_s                10001020 f i WinFallbackLookup.obj
 0001:00000040       _swscanf                   10001040 f i WinFallbackLookup.obj
 0001:00000080       _swscanf_s                 10001080 f i WinFallbackLookup.obj
 0001:000000c0       _vfprintf                  100010c0 f i WinFallbackLookup.obj
 0001:000000e0       _vfprintf_s                100010e0 f i WinFallbackLookup.obj
 0001:00000100       _vprintf                   10001100 f i WinFallbackLookup.obj
 0001:00000130       _vprintf_s                 10001130 f i WinFallbackLookup.obj
 0001:00000160       _fprintf                   10001160 f i WinFallbackLookup.obj
 0001:000001a0       _fprintf_s                 100011a0 f i WinFallbackLookup.obj
 0001:000001e0       _printf                    100011e0 f i WinFallbackLookup.obj
 0001:00000220       _printf_s                  10001220 f i WinFallbackLookup.obj
 0001:00000260       _vfscanf                   10001260 f i WinFallbackLookup.obj
 0001:00000280       _vfscanf_s                 10001280 f i WinFallbackLookup.obj
 0001:000002a0       _vscanf                    100012a0 f i WinFallbackLookup.obj
 0001:000002d0       _vscanf_s                  100012d0 f i WinFallbackLookup.obj
 0001:00000300       _fscanf                    10001300 f i WinFallbackLookup.obj
 0001:00000340       _fscanf_s                  10001340 f i WinFallbackLookup.obj
 0001:00000380       _scanf                     10001380 f i WinFallbackLookup.obj
 0001:000003c0       _scanf_s                   100013c0 f i WinFallbackLookup.obj
 0001:00000400       _vsnprintf                 10001400 f i WinFallbackLookup.obj
 0001:00000450       _vsprintf                  10001450 f i WinFallbackLookup.obj
 0001:00000470       _vsprintf_s                10001470 f i WinFallbackLookup.obj
 0001:00000490       _vsnprintf_s               10001490 f i WinFallbackLookup.obj
 0001:000004c0       _sprintf                   100014c0 f i WinFallbackLookup.obj
 0001:00000500       _sprintf_s                 10001500 f i WinFallbackLookup.obj
 0001:00000540       _snprintf                  10001540 f i WinFallbackLookup.obj
 0001:00000580       _vsscanf                   10001580 f i WinFallbackLookup.obj
 0001:000005a0       _vsscanf_s                 100015a0 f i WinFallbackLookup.obj
 0001:000005c0       _sscanf                    100015c0 f i WinFallbackLookup.obj
 0001:00000600       _sscanf_s                  10001600 f i WinFallbackLookup.obj
 0001:00000660       _vfwprintf                 10001660 f i WinFallbackLookup.obj
 0001:00000680       _vfwprintf_s               10001680 f i WinFallbackLookup.obj
 0001:000006a0       _vwprintf                  100016a0 f i WinFallbackLookup.obj
 0001:000006d0       _vwprintf_s                100016d0 f i WinFallbackLookup.obj
 0001:00000700       _fwprintf                  10001700 f i WinFallbackLookup.obj
 0001:00000740       _fwprintf_s                10001740 f i WinFallbackLookup.obj
 0001:00000780       _wprintf                   10001780 f i WinFallbackLookup.obj
 0001:000007c0       _wprintf_s                 100017c0 f i WinFallbackLookup.obj
 0001:00000800       _vfwscanf                  10001800 f i WinFallbackLookup.obj
 0001:00000820       _vfwscanf_s                10001820 f i WinFallbackLookup.obj
 0001:00000840       _vwscanf                   10001840 f i WinFallbackLookup.obj
 0001:00000870       _vwscanf_s                 10001870 f i WinFallbackLookup.obj
 0001:000008a0       _fwscanf                   100018a0 f i WinFallbackLookup.obj
 0001:000008e0       _fwscanf_s                 100018e0 f i WinFallbackLookup.obj
 0001:00000920       _wscanf                    10001920 f i WinFallbackLookup.obj
 0001:00000960       _wscanf_s                  10001960 f i WinFallbackLookup.obj
 0001:000009a0       _vswprintf                 100019a0 f i WinFallbackLookup.obj
 0001:000009c0       _vswprintf_s               100019c0 f i WinFallbackLookup.obj
 0001:000009e0       _swprintf                  100019e0 f i WinFallbackLookup.obj
 0001:00000a20       _swprintf_s                10001a20 f i WinFallbackLookup.obj
 0001:00000a60       ___local_stdio_printf_options 10001a60 f i WinFallbackLookup.obj
 0001:00000a70       ___local_stdio_scanf_options 10001a70 f i WinFallbackLookup.obj
 0001:00000a80       __vfprintf_l               10001a80 f i WinFallbackLookup.obj
 0001:00000ab0       __vfprintf_s_l             10001ab0 f i WinFallbackLookup.obj
 0001:00000ae0       __vfscanf_l                10001ae0 f i WinFallbackLookup.obj
 0001:00000b10       __vfscanf_s_l              10001b10 f i WinFallbackLookup.obj
 0001:00000b40       __vfwprintf_l              10001b40 f i WinFallbackLookup.obj
 0001:00000b70       __vfwprintf_s_l            10001b70 f i WinFallbackLookup.obj
 0001:00000ba0       __vfwscanf_l               10001ba0 f i WinFallbackLookup.obj
 0001:00000bd0       __vfwscanf_s_l             10001bd0 f i WinFallbackLookup.obj
 0001:00000c00       __vsnprintf_l              10001c00 f i WinFallbackLookup.obj
 0001:00000c60       __vsnprintf_s_l            10001c60 f i WinFallbackLookup.obj
 0001:00000cc0       __vsprintf_l               10001cc0 f i WinFallbackLookup.obj
 0001:00000ce0       __vsprintf_s_l             10001ce0 f i WinFallbackLookup.obj
 0001:00000d30       __vsscanf_l                10001d30 f i WinFallbackLookup.obj
 0001:00000d60       __vsscanf_s_l              10001d60 f i WinFallbackLookup.obj
 0001:00000d90       __vswprintf_c_l            10001d90 f i WinFallbackLookup.obj
 0001:00000de0       __vswprintf_s_l            10001de0 f i WinFallbackLookup.obj
 0001:00000e30       __vswscanf_l               10001e30 f i WinFallbackLookup.obj
 0001:00000e60       __vswscanf_s_l             10001e60 f i WinFallbackLookup.obj
 0001:000011cf       __DllMainCRTStartup@12     100021cf f   MSVCRT:dll_dllmain.obj
 0001:0000123f       ___security_init_cookie    1000223f f   MSVCRT:gs_support.obj
 0001:0000128a       _DllMain@12                1000228a f   MSVCRT:dll_dllmain_stub.obj
 0001:000012ac       ?__scrt_initialize_type_info@@YAXXZ 100022ac f   MSVCRT:tncleanup.obj
 0001:000012b8       ?__scrt_uninitialize_type_info@@YAXXZ 100022b8 f   MSVCRT:tncleanup.obj
 0001:000012c4       ___scrt_initialize_default_local_stdio_options 100022c4 f   MSVCRT:default_local_stdio_options.obj
 0001:00001325       ___scrt_acquire_startup_lock 10002325 f   MSVCRT:utility.obj
 0001:00001357       ___scrt_dllmain_after_initialize_c 10002357 f   MSVCRT:utility.obj
 0001:00001382       ___scrt_dllmain_before_initialize_c 10002382 f   MSVCRT:utility.obj
 0001:00001390       ___scrt_dllmain_crt_thread_attach 10002390 f   MSVCRT:utility.obj
 0001:000013af       ___scrt_dllmain_crt_thread_detach 100023af f   MSVCRT:utility.obj
 0001:000013bc       ___scrt_dllmain_exception_filter 100023bc f   MSVCRT:utility.obj
 0001:000013f0       ___scrt_dllmain_uninitialize_c 100023f0 f   MSVCRT:utility.obj
 0001:00001413       ___scrt_dllmain_uninitialize_critical 10002413 f   MSVCRT:utility.obj
 0001:00001420       ___scrt_initialize_crt     10002420 f   MSVCRT:utility.obj
 0001:00001459       ___scrt_initialize_onexit_tables 10002459 f   MSVCRT:utility.obj
 0001:000014e0       ___scrt_is_nonwritable_in_current_image 100024e0 f   MSVCRT:utility.obj
 0001:00001574       ___scrt_release_startup_lock 10002574 f   MSVCRT:utility.obj
 0001:00001591       ___scrt_uninitialize_crt   10002591 f   MSVCRT:utility.obj
 0001:000015b9       ___scrt_get_dyn_tls_init_callback 100025b9 f   MSVCRT:dyn_tls_init.obj
 0001:000015bf       ___scrt_fastfail           100025bf f   MSVCRT:utility_desktop.obj
 0001:000016da       __crt_debugger_hook        100026da f   MSVCRT:utility_desktop.obj
 0001:000016e2       __RTC_Initialize           100026e2 f   MSVCRT:initsect.obj
 0001:0000170e       __RTC_Terminate            1000270e f   MSVCRT:initsect.obj
 0001:00001740       __SEH_prolog4              10002740 f   MSVCRT:sehprolg4.obj
 0001:00001785       __except_handler4          10002785 f   MSVCRT:chandler4gs.obj
 0001:000017b4       @_guard_check_icall_nop@4  100027b4 f i MSVCRT:guard_support.obj
 0001:000017b7       ___isa_available_init      100027b7 f   MSVCRT:cpu_disp.obj
 0001:0000198b       __get_startup_argv_mode    1000298b f   MSVCRT:argv_mode.obj
 0001:0000198f       ___scrt_is_ucrt_dll_in_use 1000298f f   MSVCRT:ucrt_detection.obj
 0001:0000199b       @__security_check_cookie@4 1000299b f   MSVCRT:secchk.obj
 0001:000019a9       ___raise_securityfailure   100029a9 f   MSVCRT:gs_report.obj
 0001:000019d1       ___report_gsfailure        100029d1 f   MSVCRT:gs_report.obj
 0001:00001acb       ___std_type_info_destroy_list 10002acb f   vcruntime:VCRUNTIME140.dll
 0001:00001ad1       _memset                    10002ad1 f   vcruntime:VCRUNTIME140.dll
 0001:00001ad7       __except_handler4_common   10002ad7 f   vcruntime:VCRUNTIME140.dll
 0001:00001add       __initterm                 10002add f   ucrt:api-ms-win-crt-runtime-l1-1-0.dll
 0001:00001ae3       __initterm_e               10002ae3 f   ucrt:api-ms-win-crt-runtime-l1-1-0.dll
 0001:00001ae9       __seh_filter_dll           10002ae9 f   ucrt:api-ms-win-crt-runtime-l1-1-0.dll
 0001:00001aef       __configure_narrow_argv    10002aef f   ucrt:api-ms-win-crt-runtime-l1-1-0.dll
 0001:00001af5       __initialize_narrow_environment 10002af5 f   ucrt:api-ms-win-crt-runtime-l1-1-0.dll
 0001:00001afb       __initialize_onexit_table  10002afb f   ucrt:api-ms-win-crt-runtime-l1-1-0.dll
 0001:00001b01       __execute_onexit_table     10002b01 f   ucrt:api-ms-win-crt-runtime-l1-1-0.dll
 0001:00001b07       __cexit                    10002b07 f   ucrt:api-ms-win-crt-runtime-l1-1-0.dll
 0001:00001b0d       ___acrt_initialize         10002b0d f   MSVCRT:ucrt_stubs.obj
 0001:00001b0d       ___acrt_thread_attach      10002b0d f   MSVCRT:ucrt_stubs.obj
 0001:00001b0d       ___acrt_thread_detach      10002b0d f   MSVCRT:ucrt_stubs.obj
 0001:00001b0d       ___acrt_uninitialize       10002b0d f   MSVCRT:ucrt_stubs.obj
 0001:00001b0d       ___acrt_uninitialize_critical 10002b0d f   MSVCRT:ucrt_stubs.obj
 0001:00001b0d       ___scrt_stub_for_acrt_initialize 10002b0d f   MSVCRT:ucrt_stubs.obj
 0001:00001b0d       ___scrt_stub_for_acrt_thread_attach 10002b0d f   MSVCRT:ucrt_stubs.obj
 0001:00001b0d       ___scrt_stub_for_acrt_thread_detach 10002b0d f   MSVCRT:ucrt_stubs.obj
 0001:00001b0d       ___scrt_stub_for_acrt_uninitialize 10002b0d f   MSVCRT:ucrt_stubs.obj
 0001:00001b0d       ___scrt_stub_for_acrt_uninitialize_critical 10002b0d f   MSVCRT:ucrt_stubs.obj
 0001:00001b0d       ___vcrt_initialize         10002b0d f   MSVCRT:ucrt_stubs.obj
 0001:00001b0d       ___vcrt_thread_attach      10002b0d f   MSVCRT:ucrt_stubs.obj
 0001:00001b0d       ___vcrt_thread_detach      10002b0d f   MSVCRT:ucrt_stubs.obj
 0001:00001b0d       ___vcrt_uninitialize       10002b0d f   MSVCRT:ucrt_stubs.obj
 0001:00001b0d       ___vcrt_uninitialize_critical 10002b0d f   MSVCRT:ucrt_stubs.obj
 0001:00001b10       ___scrt_stub_for_is_c_termination_complete 10002b10 f   MSVCRT:ucrt_stubs.obj
 0001:00001b10       __is_c_termination_complete 10002b10 f   MSVCRT:ucrt_stubs.obj
 0001:00001b13       __filter_x86_sse2_floating_point_exception 10002b13 f   MSVCRT:x86_exception_filter.obj
 0001:00001b13       __filter_x86_sse2_floating_point_exception_default 10002b13 f   MSVCRT:x86_exception_filter.obj
 0002:00000000       __imp__QueryPerformanceCounter@4 10003000     kernel32:KERNEL32.dll
 0002:00000004       __imp__GetCurrentProcessId@0 10003004     kernel32:KERNEL32.dll
 0002:00000008       __imp__GetCurrentThreadId@0 10003008     kernel32:KERNEL32.dll
 0002:0000000c       __imp__GetSystemTimeAsFileTime@4 1000300c     kernel32:KERNEL32.dll
 0002:00000010       __imp__DisableThreadLibraryCalls@4 10003010     kernel32:KERNEL32.dll
 0002:00000014       __imp__InitializeSListHead@4 10003014     kernel32:KERNEL32.dll
 0002:00000018       __imp__IsDebuggerPresent@0 10003018     kernel32:KERNEL32.dll
 0002:0000001c       __imp__UnhandledExceptionFilter@4 1000301c     kernel32:KERNEL32.dll
 0002:00000020       __imp__SetUnhandledExceptionFilter@4 10003020     kernel32:KERNEL32.dll
 0002:00000024       __imp__IsProcessorFeaturePresent@4 10003024     kernel32:KERNEL32.dll
 0002:00000028       __imp__GetCurrentProcess@0 10003028     kernel32:KERNEL32.dll
 0002:0000002c       __imp__TerminateProcess@8  1000302c     kernel32:KERNEL32.dll
 0002:00000030       \177KERNEL32_NULL_THUNK_DATA 10003030     kernel32:KERNEL32.dll
 0002:00000034       __imp____std_type_info_destroy_list 10003034     vcruntime:VCRUNTIME140.dll
 0002:00000038       __imp__memset              10003038     vcruntime:VCRUNTIME140.dll
 0002:0000003c       __imp___except_handler4_common 1000303c     vcruntime:VCRUNTIME140.dll
 0002:00000040       \177VCRUNTIME140_NULL_THUNK_DATA 10003040     vcruntime:VCRUNTIME140.dll
 0002:00000044       __imp___cexit              10003044     ucrt:api-ms-win-crt-runtime-l1-1-0.dll
 0002:00000048       __imp___initterm_e         10003048     ucrt:api-ms-win-crt-runtime-l1-1-0.dll
 0002:0000004c       __imp___execute_onexit_table 1000304c     ucrt:api-ms-win-crt-runtime-l1-1-0.dll
 0002:00000050       __imp___initialize_onexit_table 10003050     ucrt:api-ms-win-crt-runtime-l1-1-0.dll
 0002:00000054       __imp___initialize_narrow_environment 10003054     ucrt:api-ms-win-crt-runtime-l1-1-0.dll
 0002:00000058       __imp___configure_narrow_argv 10003058     ucrt:api-ms-win-crt-runtime-l1-1-0.dll
 0002:0000005c       __imp___seh_filter_dll     1000305c     ucrt:api-ms-win-crt-runtime-l1-1-0.dll
 0002:00000060       __imp___initterm           10003060     ucrt:api-ms-win-crt-runtime-l1-1-0.dll
 0002:00000064       \177api-ms-win-crt-runtime-l1-1-0_NULL_THUNK_DATA 10003064     ucrt:api-ms-win-crt-runtime-l1-1-0.dll
 0002:00000068       __imp____stdio_common_vsscanf 10003068     ucrt:api-ms-win-crt-stdio-l1-1-0.dll
 0002:0000006c       __imp____acrt_iob_func     1000306c     ucrt:api-ms-win-crt-stdio-l1-1-0.dll
 0002:00000070       __imp____stdio_common_vsnprintf_s 10003070     ucrt:api-ms-win-crt-stdio-l1-1-0.dll
 0002:00000074       __imp____stdio_common_vsprintf_s 10003074     ucrt:api-ms-win-crt-stdio-l1-1-0.dll
 0002:00000078       __imp____stdio_common_vsprintf 10003078     ucrt:api-ms-win-crt-stdio-l1-1-0.dll
 0002:0000007c       __imp____stdio_common_vfscanf 1000307c     ucrt:api-ms-win-crt-stdio-l1-1-0.dll
 0002:00000080       __imp____stdio_common_vfprintf_s 10003080     ucrt:api-ms-win-crt-stdio-l1-1-0.dll
 0002:00000084       __imp____stdio_common_vfprintf 10003084     ucrt:api-ms-win-crt-stdio-l1-1-0.dll
 0002:00000088       __imp____stdio_common_vswscanf 10003088     ucrt:api-ms-win-crt-stdio-l1-1-0.dll
 0002:0000008c       __imp____stdio_common_vswprintf_s 1000308c     ucrt:api-ms-win-crt-stdio-l1-1-0.dll
 0002:00000090       __imp____stdio_common_vfwscanf 10003090     ucrt:api-ms-win-crt-stdio-l1-1-0.dll
 0002:00000094       __imp____stdio_common_vfwprintf_s 10003094     ucrt:api-ms-win-crt-stdio-l1-1-0.dll
 0002:00000098       __imp____stdio_common_vfwprintf 10003098     ucrt:api-ms-win-crt-stdio-l1-1-0.dll
 0002:0000009c       __imp____stdio_common_vswprintf 1000309c     ucrt:api-ms-win-crt-stdio-l1-1-0.dll
 0002:000000a0       \177api-ms-win-crt-stdio-l1-1-0_NULL_THUNK_DATA 100030a0     ucrt:api-ms-win-crt-stdio-l1-1-0.dll
 0002:000000a4       __imp___gmtime64           100030a4     ucrt:api-ms-win-crt-time-l1-1-0.dll
 0002:000000a8       \177api-ms-win-crt-time-l1-1-0_NULL_THUNK_DATA 100030a8     ucrt:api-ms-win-crt-time-l1-1-0.dll
 0002:000000ac       ___guard_check_icall_fptr  100030ac     MSVCRT:guard_support.obj
 0002:000000b0       ___castguard_check_failure_os_handled_fptr 100030b0     MSVCRT:guard_support.obj
 0002:000000b4       ___xc_a                    100030b4     MSVCRT:initializers.obj
 0002:000000b8       ___xc_z                    100030b8     MSVCRT:initializers.obj
 0002:000000bc       ___xi_a                    100030bc     MSVCRT:initializers.obj
 0002:000000c0       ___xi_z                    100030c0     MSVCRT:initializers.obj
 0002:000000c4       ___xp_a                    100030c4     MSVCRT:initializers.obj
 0002:000000c8       ___xp_z                    100030c8     MSVCRT:initializers.obj
 0002:000000cc       ___xt_a                    100030cc     MSVCRT:initializers.obj
 0002:000000d0       ___xt_z                    100030d0     MSVCRT:initializers.obj
 0002:000000d8       __pDefaultRawDllMain       100030d8     MSVCRT:dll_dllmain.obj
 0002:000000d8       __pRawDllMain              100030d8     MSVCRT:dll_dllmain.obj
 0002:000000e8       __load_config_used         100030e8     MSVCRT:loadcfg.obj
 0002:00000240       ___safe_se_handler_table   10003240     <linker-defined>
 0002:00000244       ___volatile_metadata       10003244     <linker-defined>
 0002:00000548       ___rtc_iaa                 10003548     MSVCRT:initsect.obj
 0002:0000054c       ___rtc_izz                 1000354c     MSVCRT:initsect.obj
 0002:00000550       ___rtc_taa                 10003550     MSVCRT:initsect.obj
 0002:00000554       ___rtc_tzz                 10003554     MSVCRT:initsect.obj
 0002:00000630       __IMPORT_DESCRIPTOR_KERNEL32 10003630     kernel32:KERNEL32.dll
 0002:00000644       __IMPORT_DESCRIPTOR_VCRUNTIME140 10003644     vcruntime:VCRUNTIME140.dll
 0002:00000658       __IMPORT_DESCRIPTOR_api-ms-win-crt-stdio-l1-1-0 10003658     ucrt:api-ms-win-crt-stdio-l1-1-0.dll
 0002:0000066c       __IMPORT_DESCRIPTOR_api-ms-win-crt-time-l1-1-0 1000366c     ucrt:api-ms-win-crt-time-l1-1-0.dll
 0002:00000680       __IMPORT_DESCRIPTOR_api-ms-win-crt-runtime-l1-1-0 10003680     ucrt:api-ms-win-crt-runtime-l1-1-0.dll
 0002:00000694       __NULL_IMPORT_DESCRIPTOR   10003694     kernel32:KERNEL32.dll
 0003:00000000       _funcs                     10004000     WinFallbackLookup.obj
 0003:000000d0       ___scrt_native_dllmain_reason 100040d0     MSVCRT:utility.obj
 0003:000000e0       ___security_cookie_complement 100040e0     MSVCRT:gs_cookie.obj
 0003:000000e4       ___security_cookie         100040e4     MSVCRT:gs_cookie.obj
 0003:000000e8       ___isa_enabled             100040e8     MSVCRT:cpu_disp.obj
 0003:000000ec       ___scrt_ucrt_dll_is_in_use 100040ec     MSVCRT:ucrt_stubs.obj
 0003:000000f8       ?__type_info_root_node@@3U__type_info_node@@A 100040f8     MSVCRT:tncleanup.obj
 0003:00000100       ___scrt_current_native_startup_state 10004100     MSVCRT:utility.obj
 0003:00000104       ___scrt_native_startup_lock 10004104     MSVCRT:utility.obj
 0003:00000124       ___scrt_debugger_hook_flag 10004124     MSVCRT:utility_desktop.obj
 0003:00000128       ___isa_available           10004128     MSVCRT:cpu_disp.obj
 0003:0000012c       ___favor                   1000412c     MSVCRT:cpu_disp.obj
 0003:00000450       ?_OptionsStorage@?1??__local_stdio_scanf_options@@9@9 10004450     <common>
 0003:00000458       ?_OptionsStorage@?1??__local_stdio_printf_options@@9@9 10004458     <common>
 0003:00000460       ___dyn_tls_init_callback   10004460     <common>

 entry point at        0001:000011cf

 Static symbols

 0000:ffff9000       .debug$S                   10000000     WinFallbackLookup.exp
 0000:ffff9000       .debug$S                   10000000     vcruntime:VCRUNTIME140.dll
 0000:ffff9000       .debug$S                   10000000     vcruntime:VCRUNTIME140.dll
 0000:ffff9000       .debug$S                   10000000     vcruntime:VCRUNTIME140.dll
 0000:ffff9000       .debug$S                   10000000     vcruntime:VCRUNTIME140.dll
 0000:ffff9000       .debug$S                   10000000     vcruntime:VCRUNTIME140.dll
 0000:ffff9000       .debug$S                   10000000     ucrt:api-ms-win-crt-runtime-l1-1-0.dll
 0000:ffff9000       .debug$S                   10000000     ucrt:api-ms-win-crt-runtime-l1-1-0.dll
 0000:ffff9000       .debug$S                   10000000     ucrt:api-ms-win-crt-runtime-l1-1-0.dll
 0000:ffff9000       .debug$S                   10000000     ucrt:api-ms-win-crt-runtime-l1-1-0.dll
 0000:ffff9000       .debug$S                   10000000     ucrt:api-ms-win-crt-runtime-l1-1-0.dll
 0000:ffff9000       .debug$S                   10000000     ucrt:api-ms-win-crt-runtime-l1-1-0.dll
 0000:ffff9000       .debug$S                   10000000     ucrt:api-ms-win-crt-runtime-l1-1-0.dll
 0000:ffff9000       .debug$S                   10000000     ucrt:api-ms-win-crt-runtime-l1-1-0.dll
 0000:ffff9000       .debug$S                   10000000     ucrt:api-ms-win-crt-runtime-l1-1-0.dll
 0000:ffff9000       .debug$S                   10000000     ucrt:api-ms-win-crt-runtime-l1-1-0.dll
 0000:ffff9000       .debug$S                   10000000     ucrt:api-ms-win-crt-runtime-l1-1-0.dll
 0000:ffff9000       .debug$S                   10000000     ucrt:api-ms-win-crt-runtime-l1-1-0.dll
 0000:ffff9000       .debug$S                   10000000     ucrt:api-ms-win-crt-stdio-l1-1-0.dll
 0000:ffff9000       .debug$S                   10000000     ucrt:api-ms-win-crt-stdio-l1-1-0.dll
 0000:ffff9000       .debug$S                   10000000     ucrt:api-ms-win-crt-stdio-l1-1-0.dll
 0000:ffff9000       .debug$S                   10000000     ucrt:api-ms-win-crt-stdio-l1-1-0.dll
 0000:ffff9000       .debug$S                   10000000     ucrt:api-ms-win-crt-stdio-l1-1-0.dll
 0000:ffff9000       .debug$S                   10000000     ucrt:api-ms-win-crt-stdio-l1-1-0.dll
 0000:ffff9000       .debug$S                   10000000     ucrt:api-ms-win-crt-stdio-l1-1-0.dll
 0000:ffff9000       .debug$S                   10000000     ucrt:api-ms-win-crt-stdio-l1-1-0.dll
 0000:ffff9000       .debug$S                   10000000     ucrt:api-ms-win-crt-stdio-l1-1-0.dll
 0000:ffff9000       .debug$S                   10000000     ucrt:api-ms-win-crt-stdio-l1-1-0.dll
 0000:ffff9000       .debug$S                   10000000     ucrt:api-ms-win-crt-stdio-l1-1-0.dll
 0000:ffff9000       .debug$S                   10000000     ucrt:api-ms-win-crt-stdio-l1-1-0.dll
 0000:ffff9000       .debug$S                   10000000     ucrt:api-ms-win-crt-stdio-l1-1-0.dll
 0000:ffff9000       .debug$S                   10000000     ucrt:api-ms-win-crt-stdio-l1-1-0.dll
 0000:ffff9000       .debug$S                   10000000     ucrt:api-ms-win-crt-time-l1-1-0.dll
 0000:ffff9000       .debug$S                   10000000     kernel32:KERNEL32.dll
 0000:ffff9000       .debug$S                   10000000     kernel32:KERNEL32.dll
 0000:ffff9000       .debug$S                   10000000     kernel32:KERNEL32.dll
 0000:ffff9000       .debug$S                   10000000     kernel32:KERNEL32.dll
 0000:ffff9000       .debug$S                   10000000     kernel32:KERNEL32.dll
 0000:ffff9000       .debug$S                   10000000     kernel32:KERNEL32.dll
 0000:ffff9000       .debug$S                   10000000     kernel32:KERNEL32.dll
 0000:ffff9000       .debug$S                   10000000     kernel32:KERNEL32.dll
 0000:ffff9000       .debug$S                   10000000     kernel32:KERNEL32.dll
 0000:ffff9000       .debug$S                   10000000     kernel32:KERNEL32.dll
 0000:ffff9000       .debug$S                   10000000     kernel32:KERNEL32.dll
 0000:ffff9000       .debug$S                   10000000     kernel32:KERNEL32.dll
 0000:ffff9000       .debug$S                   10000000     kernel32:KERNEL32.dll
 0000:ffff9000       .debug$S                   10000000     kernel32:KERNEL32.dll
 0001:00000640       _gmtime                    10001640 f   WinFallbackLookup.obj
 0001:00000e8f       ?dllmain_crt_dispatch@@YGHQAUHINSTANCE__@@KQAX@Z 10001e8f f   MSVCRT:dll_dllmain.obj
 0001:00000ee2       ?dllmain_crt_process_attach@@YAHQAUHINSTANCE__@@QAX@Z 10001ee2 f   MSVCRT:dll_dllmain.obj
 0001:00000fe9       ?dllmain_crt_process_detach@@YAH_N@Z 10001fe9 f   MSVCRT:dll_dllmain.obj
 0001:00001099       ?dllmain_dispatch@@YAHQAUHINSTANCE__@@KQAX@Z 10002099 f   MSVCRT:dll_dllmain.obj
 0001:000011a4       ?dllmain_raw@@YGHQAUHINSTANCE__@@KQAX@Z 100021a4 f   MSVCRT:dll_dllmain.obj
 0001:000011f2       ___get_entropy             100021f2 f   MSVCRT:gs_support.obj
 0001:000012e1       ?find_pe_section@@YAPAU_IMAGE_SECTION_HEADER@@QAEI@Z 100022e1 f   MSVCRT:utility.obj
 0001:00001740       $$000000                   10002740     MSVCRT:sehprolg4.obj
 0002:000000dc       _GS_ExceptionPointers      100030dc     MSVCRT:gs_report.obj
 0002:00000558       __sehtable$?dllmain_crt_process_attach@@YAHQAUHINSTANCE__@@QAX@Z 10003558     MSVCRT:dll_dllmain.obj
 0002:00000578       __sehtable$?dllmain_crt_process_detach@@YAH_N@Z 10003578     MSVCRT:dll_dllmain.obj
 0002:000005a0       __sehtable$?dllmain_dispatch@@YAHQAUHINSTANCE__@@KQAX@Z 100035a0     MSVCRT:dll_dllmain.obj
 0002:000005c0       __sehtable$___scrt_is_nonwritable_in_current_image 100035c0     MSVCRT:utility.obj
 0002:000005e0       .edata                     100035e0     WinFallbackLookup.exp
 0002:00000608       rgpv                       10003608     WinFallbackLookup.exp
 0002:0000060c       rgszName                   1000360c     WinFallbackLookup.exp
 0002:00000610       rgwOrd                     10003610     WinFallbackLookup.exp
 0002:00000612       szName                     10003612     WinFallbackLookup.exp
 0002:00000628       $N00001                    10003628     WinFallbackLookup.exp
 0002:00000878       .idata$6                   10003878     kernel32:KERNEL32.dll
 0002:000008ca       .idata$6                   100038ca     vcruntime:VCRUNTIME140.dll
 0002:00000b06       .idata$6                   10003b06     ucrt:api-ms-win-crt-stdio-l1-1-0.dll
 0002:00000b26       .idata$6                   10003b26     ucrt:api-ms-win-crt-time-l1-1-0.dll
 0002:00000b46       .idata$6                   10003b46     ucrt:api-ms-win-crt-runtime-l1-1-0.dll
 0003:000000f0       ?__proc_attached@@3HA      100040f0     MSVCRT:dll_dllmain.obj
 0003:00000108       ?is_initialized_as_dll@@3_NA 10004108     MSVCRT:utility.obj
 0003:00000109       ?module_local_atexit_table_initialized@@3_NA 10004109     MSVCRT:utility.obj
 0003:0000010c       ?module_local_atexit_table@@3U_onexit_table_t@@A 1000410c     MSVCRT:utility.obj
 0003:00000118       ?module_local_at_quick_exit_table@@3U_onexit_table_t@@A 10004118     MSVCRT:utility.obj
 0003:00000130       _GS_ExceptionRecord        10004130     MSVCRT:gs_report.obj
 0003:00000180       _GS_ContextRecord          10004180     MSVCRT:gs_report.obj
 0004:00000060       $R000000                   10005060     WinFallbackLookup.dll.res
